:020000040000FA
:1000000000008A150A168C2EFF3FFF3FFF3FFF3F7F
:100010000406031D052864000034FF3FFF3FFF3F37
:10002000FF3FFF3FFF3FFF3FFF3FFF3FFF3FFF3FE0
:10003000FF3FFF3FFF3FFF3FFF3FFF3FFF3FFF3FD0
:10004000FF3FFF3FFF3FFF3FFF3FFF3FFF3FFF3FC0
:10005000FF3FFF3FFF3FFF3FFF3FFF3FFF3FFF3FB0
:100E1000FF3F8301A100A4011A2FA301A201A20A8E
:100E2000CF302202031C0F2FA30A0F302302031C12
:100E30000E2FA40A21082402031808000D2F830195
:100E4000A2009F00A401252FA40A10302402031C35
:100E5000242F1F151F192A2F1E08A3001F10A401DD
:100E6000103024020318362FA40A302F230808005C
:100E70007F3083120313A000FF30831685008601A4
:100E800087018312071187108716071460308316B5
:100E90008800FF30831288008316890102309F008A
:100EA00081301F27F00080307002031C602FA130BA
:100EB0001F27F00080307002031C602F6427632F0F
:100EC0002008AE27602F0028FF308301880008101B
:100ED000E83009278810E83009270811E830092789
:100EE0008811E83009270812E8300927FF30880008
:100EF0008714071507148716A1301F27F0007F30CD
:100F0000700203188B2F08120710871290300927E0
:100F100087169030092781301F27F0007F3070023C
:100F200003189A2F0810071087129030092707140A
:100F300090300927081F881AA12F881088110A30BD
:100F4000752F081BA72F881488110711AC2F881A3A
:100F5000762F8810881587106430752F8301A100C3
:100F600081301F27F000210870020318B92F0814E0
:100F7000BA2F081089301F27F000210870020318CB
:100F8000C32F8814C42F881091301F27F000210828
:100F900070020318CD2F0815CE2F081199301F2786
:100FA000F000210870020318D72F8815D82F881158
:100FB000A1301F27F000210870020318E12F081646
:100FC000E22F081287140715071487160818EA2F4E
:100FD000071008008818EE2F871008000819F52F51
:100FE000871407150714871608008819F92F0711A9
:100FF0000800081AFD2F8712080087100711080043
:10100000FF3FFF3FFF3FFF3FFF3FFF3FFF3FFF3FF0
:10101000FF3FFF3FFF3FFF3FFF3FFF3FFF3FFF3FE0
:10102000FF3FFF3FFF3FFF3FFF3FFF3FFF3FFF3FD0
:10103000FF3FFF3FFF3FFF3FFF3FFF3FFF3FFF3FC0
:103D00008A150A16802E8A0120308400253008206A
:103D1000382F04068001840A031E832E90309800F9
:103D20008316181598161F30990083120330FA0075
:103D3000313090000C14F026EA3A031DB32EFA013C
:103D4000BA2EF026F900E33A0319BC2E7908EA3AB4
:103D50000319BA2E7908ED3A031DA12EE430EB26A3
:103D60000330FA00F026900198018316980183121F
:103D70008C01832EEB30E92EF026F600F026F500BC
:103D8000F026F100FB00F026F300F201213083124F
:103D9000031376020319D52E75080339FC00FD00C4
:103DA0000310FC0D20307C07D62E20308400F02636
:103DB0008000F207840AFB0BD72E72087306E830E6
:103DC000031DE92EE730EB2602270038E430031903
:103DD000E530EB26A12E64000C1EEB2E99000800A6
:103DE00064007A080319FE2E0C1CFE2E1010FA0B2C
:103DF000FA2E00340C100B308F0010148C1EF02E95
:103E00001A080800213076020319542F831603176D
:103E10008C17831203137508FC3903178D000313E5
:103E2000760803178F002030840003137D080319E0
:103E30002C2F831603170C140000000083120E08A9
:103E40008000840A0C088000840A8D0A0313FD0395
:103E5000F503F10AF10A152F7108FC00203E8400D9
:103E60000310FC0C760803178F0003137508031763
:103E70008D0003137C0803178D0703198F0A03179E
:103E80000D0803390319542F83160C140000000089
:103E900083120E088000840A0C088000840A8D0AB0
:103EA0000313F10AF10A3F2F7508F7007608F800AE
:103EB000FB010230F40071087B02031801347B0817
:103EC000203E840021307802031783160319722FD5
:103ED0008C1783011E307802803003197702031893
:103EE000BA2F742F8C138301770803178D000313E7
:103EF0007808031D892F083077020318892F0317CC
:103F000083168C1F862F831284308D0783011E3009
:103F10008A2F780803178F0000088E00840A000893
:103F20008C0083160C1555308D00AA308D008C1432
:103F3000000000008301831603178C1BC22F83121D
:103F4000031364000D1EA12F0D12831603170C110D
:103F50000C14000000008312840300080E06031DE9
:103F6000B62F840A00080C060319BA2F8301F40B3C
:103F70005B2F0034831203130230FB07F70A031987
:103F8000F80A592F831203130D12831603170C110D
:103F9000831203170D080339033C031DBA2F0330A6
:103FA0008D02831203130430FC00073084020000EA
:103FB000831603170C14000000000000000000002E
:103FC00000000008831203170E06031DEC2F840A5D
:103FD00000080C060319F32F83120313FC30F705B6
:103FE0000630FB02B62F831203178D0A840A831250
:103FF0000313FC0BD72FBA2FFF3FFF3FFF3FFF3FBD
:084000000200010000000000B5
:10420000FF00FF00FF00FF00FF00FF00FF00FF00B6
:10421000FF00FF00FF00FF00FF00FF00FF00FF00A6
:10422000FF00FF00FF00FF00FF00FF00FF00FF0096
:10423000FF00FF00FF00FF00FF00FF00FF00FF0086
:10424000FF00FF00FF00FF00FF00FF00FF00FF0076
:10425000FF00FF00FF00FF00FF00FF00FF00FF0066
:10426000FF00FF00FF00FF00FF00FF00FF00FF0056
:10427000FF00FF00FF00FF00FF00FF00FF00FF0046
:10428000FF00FF00FF00FF00FF00FF00FF00FF0036
:10429000FF00FF00FF00FF00FF00FF00FF00FF0026
:1042A000FF00FF00FF00FF00FF00FF00FF00FF0016
:1042B000FF00FF00FF00FF00FF00FF00FF00FF0006
:1042C000FF00FF00FF00FF00FF00FF00FF00FF00F6
:1042D000FF00FF00FF00FF00FF00FF00FF00FF00E6
:1042E000FF00FF00FF00FF00FF00FF00FF00FF00D6
:1042F000FF00FF00FF00FF00FF00FF00FF00FF00C6
:10430000FF00FF00FF00FF00FF00FF00FF00FF00B5
:10431000FF00FF00FF00FF00FF00FF00FF00FF00A5
:10432000FF00FF00FF00FF00FF00FF00FF00FF0095
:10433000FF00FF00FF00FF00FF00FF00FF00FF0085
:10434000FF00FF00FF00FF00FF00FF00FF00FF0075
:10435000FF00FF00FF00FF00FF00FF00FF00FF0065
:10436000FF00FF00FF00FF00FF00FF00FF00FF0055
:10437000FF00FF00FF00FF00FF00FF00FF00FF0045
:10438000FF00FF00FF00FF00FF00FF00FF00FF0035
:10439000FF00FF00FF00FF00FF00FF00FF00FF0025
:1043A000FF00FF00FF00FF00FF00FF00FF00FF0015
:1043B000FF00FF00FF00FF00FF00FF00FF00FF0005
:1043C000FF00FF00FF00FF00FF00FF00FF00FF00F5
:1043D000FF00FF00FF00FF00FF00FF00FF00FF00E5
:1043E000FF00FF00FF00FF00FF00FF00FF00FF00D5
:1043F000FF00FF00FF00FF00FF00FF00FF00FF00C5
:00000001FF
